:1000000012C021C020C01FC01EC01DC01CC01BC00C
:100010001AC019C018C017C016C015C014C013C02C
:1000200012C011C010C011241FBECFE5D4E0DEBF46
:10003000CDBF10E0A0E6B0E001C01D92A136B1072F
:10004000E1F7B8D134C2DCCF20E030E040EA5FE035
:1000500005C0FA013197F1F72F5F3F4F2817390795
:10006000C0F308958FB9779BFECF0895E199FECF35
:100070009FBB8EBB6DBBE29AE19A0895E199FECFDA
:100080009FBB8EBBE09A8DB3089580E49CE90197F5
:10009000F1F7C09A80E09FEF9FB9779BFECF8F5F0B
:1000A0008A30D1F7C09880E48FB9779BFECF1FB814
:1000B000779BFECF1FB8779BFECF1FB8779BFECFF5
:1000C0001FB8779BFECF85E98FB9779BFECF8FEF67
:1000D0008FB9779BFECF8FEF8FB9779BFECF8FB114
:1000E000813011F080E0089521E49FEF2FB9779BD4
:1000F000FECF1FB8779BFECF1FB8779BFECF1FB8F0
:10010000779BFECF1FB8779BFECF9FB9779BFECF23
:100110009FB9779BFECF9FB9779BFECF8FB1882386
:1001200029F781E00895DF92EF92FF920F931F93DA
:10013000CF93DF93959AC0E0D0E0CE016FEF96DFCA
:10014000219662E0C030D607C1F782E58FB9779B70
:10015000FECF1FB8779BFECF1FB8779BFECF80E8FE
:100160008FB9779BFECF1FB8779BFECF8FEF8FB9EC
:10017000779BFECF9FEF9FB9779BFECF8FB18E3FCE
:10018000D1F7E12CF0E8FF2E012D112DDD24DA94BA
:10019000DFB8779BFECF5FB1DFB8779BFECF4FB163
:1001A000DFB8779BFECF3FB1DFB8779BFECF2FB193
:1001B00080E090E0DFB8779BFECF0196A2E082302E
:1001C0009A07C1F75235E9F54934D9F53634C9F5FE
:1001D0002634B9F58091600090E0212F3327442721
:1001E0005527880F991F880F991F622F3FDF809135
:1001F000600090E0880F991F880F991F980144278D
:1002000055270196622F32DF8091600090E0880FC1
:10021000991F880F991F5527412F302F2F2D029698
:10022000622F24DF8091600090E0880F991F880F73
:10023000991F039660E01ADF809160008F5F8093C2
:10024000600080E092E0A0E0B0E0E80EF91E0A1F36
:100250001B1F90E0E91690E0F90690E009079CE387
:10026000190709F095CF8FEF91E060916000FEDEF5
:100270009598DF91CF911F910F91FF90EF90DF90B4
:100280000895982F82E58FB9779BFECF492F50E0D4
:100290009A01220F331F220F331FE199FECF3FBB7C
:1002A0002EBBE09A8DB38FB9779BFECFE199FECF3D
:1002B0002F5F3F4F3FBB2EBB21503040E09A8DB3A4
:1002C0008FB9779BFECFE199FECF440F551F440FA6
:1002D000551F4E5F5F4F5FBB4EBBE09A8DB38FB92A
:1002E000779BFECFE199FECF2D5F3F4F3FBB2EBBEB
:1002F000E09A8DB38FB9779BFECF8FEF8FB9779B45
:10030000FECF9FEF9FB9779BFECF8FB18E3FD1F786
:1003100080E090E02FEF2FB9779BFECF019632E07F
:1003200086309307C1F70895979A4FEF50E922C09E
:1003300020E030E04FB9779BFECF8FB190E09BBDBE
:100340008ABD4FB9779BFECF8FB190E099BD88BD34
:10035000849B03C0852F8A95F1F72F5F3F4F81E083
:100360002030380739F780E04FB9779BFECF8F5F99
:100370008630D1F78399DCCF089597988CE48FB9B4
:10038000779BFECF1FB8779BFECF1FB8779BFECF22
:100390001FB8779BFECF1FB8779BFECF8FEF8FB92B
:1003A000779BFECF9FEF9FB9779BFECF8FB18F3F9B
:1003B000D1F708951F93CF93DF938FEE87BB8FEF15
:1003C00084BB80EE81BB8FE182BB80E58DB991E07B
:1003D0009EB981EA8FBD9EBD80E890E09BBD8ABD3D
:1003E00099BD88BD8CE291E020E931E0F9013197B7
:1003F000F1F70197D9F749DE8823E9F380B38F310C
:1004000009F091DEE199FECF8FEF91E09FBB8EBBAB
:10041000E09A1DB3115020E040EA5FE0979A80E037
:1004200090E0FA013197F1F70196883C9105C9F700
:10043000979880E090E0FA013197F1F70196883CB7
:100440009105C9F72F5F233049F7C0EADFE08091BB
:100450006000809910C08F5F181708F480E0969AAA
:1004600020E030E0FE013197F1F72F5F3F4F283C4D
:100470003105C1F79698819912C0982F9150812F1C
:10048000911708F4892F969A20E030E0FE01319709
:10049000F1F72F5F3F4F283C3105C1F796988299BD
:1004A000D8CF80936000EDDE3FDF67DFD0CFF894D8
:0204B000FFCF7C
:00000001FF
